:030000000211E307
:03000B000200C12F
:03002B000203CB02
:03005B0002051D7E
:0300730002051370
:1000800002030406080C10182030406080020304AC
:1000900006080C101820304080FF0406080C1018C9
:1000A0002030406080A0C000000001010003020277
:1000B000010D0D040506020D0505050D06030502DB
:1000C00002C2AFC0D0C0E0205A0D302F02E473301E
:1000D000600280F90203B7306306D297D295D293BB
:1000E00085258AC25AE525F4700221AA056130608F
:1000F00013206A19758B00D0E0D0D0D297D295D258
:1001000093D2AF32D297D295D29302019AD26EC2D5
:100110006FE565601CC3E5611495654014C26ED23D
:100120006FC3E5619564500302019A756100020195
:100130009A206C14D297D295D2937401D5E0FDD257
:1001400096D294D29202019AD297D295D293E53D5B
:1001500020E22520E10D207502D296307502D2945E
:1001600002019A20E005D29202019A207502D294EF
:10017000307502D29602019A20E11520E00D20751B
:1001800002D296307502D29402019AD29202019A5A
:10019000207502D294307502D296758B00D0E0D0D3
:1001A000D0D297D295D293D2AF32D0E0D0D0D2AFC6
:1001B0003261B7E525600A207502C297307502C228
:1001C00095D29361B7E5256002C293207502D2955E
:1001D000307502D29761B7E525600A207502C29595
:1001E000307502C297207502D297307502D29561A0
:1001F000B7207502C296307502C294E525600A20C8
:100200007502C297307502C295207502C29430758E
:1002100002C296D29361B7207502C296307502C2AF
:1002200094207502C294307502C2967419D5E0FD0F
:10023000E525600A207502C297307502C295D293F7
:1002400061B7207502C296307502C294E525600A36
:10025000207502C297307502C295C292D29361B7DF
:10026000207502C296307502C294C2927419D5E00C
:10027000FDE525600A207502C297307502C295D24D
:100280009361B7C292E5256002C293207502C296BF
:10029000307502C294207502D295307502D29761F2
:1002A000B7C292207502C296307502C2947419D5F5
:1002B000E0FDE5256002C293207502D295307502FB
:1002C000D29761B7C292E5256002C293207502C23F
:1002D00094307502C296207502D295307502D2977D
:1002E00061B7C292207502C294307502C296741929
:1002F000D5E0FDE5256002C293207502D2953075E8
:1003000002D29761B7207502C294307502C296E599
:1003100025600A207502C295307502C297C29220EC
:100320007502D297307502D29561B7207502C294DA
:10033000307502C296C2927419D5E0FDE525600AB7
:10034000207502C295307502C297207502D297308F
:100350007502D29561B7207502C294307502C296BB
:10036000E525600A207502C295307502C297207596
:1003700002C296307502C294207502D2973075027F
:10038000D29561B7207502C294307502C29620756D
:1003900002C296307502C2947419D5E0FDE525605D
:1003A0000A207502C295307502C297207502D29755
:1003B000307502D29561B7E525F4F58A758B007525
:1003C0006000D25AD0E0D0D0D2AF32C2AFC0D0C0DD
:1003D000E0D2D3C2CEE528600A741F552E604915BD
:1003E00028812878007900E580307601F430E50234
:1003F00078FF53DACF20760343DA2030760343DAEE
:1004000010C2D8C269E580307601F430E50279FF88
:10041000C3E89970CE305903752818741F552E60A3
:10042000037528188858D268E52960041529813B8E
:10043000741F552E600543DA01C2D820680281CDB1
:10044000E558F8C268741F552E60367982B70431BA
:10045000C3E894F0400374F0F8E8C4540F28F87926
:1004600084B703028181C313C3138721200802C309
:0E04700013200A06C3C898F8818128F85003AB
:10047E0074FFF8C3E8955F5003E55FF8E52C54066A
:10048E00703D882230630AC3E522955C4003855C8B
:10049E00227882B60429C3E5229524401278A096CC
:1004AE00400DE52426F52450097524FF0204C0856D
:1004BE002224852425C3E524955C4003855C2520F4
:1004CE00CF09D0E0D0D0C2D3D2AF32C2CF7801E5BF
:1004DE00286008741F552E70021528C3E558940124
:1004EE004005755B0081FCE55B046002055BE55D24
:1004FE00C3240A5005755DFFA10AF55DD0E0D0D08A
:10050E00C2D3D2AF32C2AF53917FC258D2AF32C232
:10051E00AFC0D0C0E0C0F0D2D3A8FBA9FCC2D83087
:10052E006902A18053DACF20760343DA10307603C6
:10053E0043DA20D269E580307601F420E502A15439
:10054E0088268927E12053DACF20760343DA20303C
:10055E00760343DA10C2D8C269741F552E7002E1B9
:10056E00067800E580307601F430E502E106885821
:10057E00E10653DACF20760343DA2030760343DAEE
:10058E0010C269205902C13A53DACF20760343DAFA
:10059E001030760343DA20C2D8D26988538954C307
:1005AE00E89551F8E99552F9E4FB7AFAC3E894C854
:1005BE00E994005008E4D2E4FB7A0AC10DC3E89432
:1005CE0068E994015008E4D2E3FB7A0FC10DC3E849
:1005DE0094D0E994025008E4D2E2FB7A1EC10DC316
:1005EE00E894A0E994055008E4D2E1FB7A3CC10DF1
:1005FE00C3E89498E994085006E4D2E0FB7A78C3F5
:10060E00E89555FCE99556FD30E708ECF42401FC1D
:10061E00EDF4FD7557007008C3EC9A500375570141
:10062E0088558956A853A95488518952C3E89526EE
:10063E00F8E99527F9307402C1D9307302C1D93067
:10064E007202C1D2E9C313F9E813F8307102C1D2B4
:10065E00E9C313F9E813F8307002C1D2E9C313FDF0
:10066E00E813FC205918C3EC941CED9402400302CD
:10067E000706ED7009C3EC94C850030207207400FE
:10068E002077037896E624FAFEE43400FFC3EC9E4E
:10069E00FCED9FFD500678007900C1D9C3EC94FFA4
:1006AE00ED9400400678FF7900C1D9EC856CF0A47A
:1006BE00C5F0A2F733F8790040030206F578FF790A
:1006CE00000206F5E9C313F9E813F830740EE96079
:1006DE000278FFC3E81338F8E43400F9C3E894FF56
:1006EE00E99400400278FF8858D268205902E1064A
:1006FE00741FF4552E4BF52E752818741F552E7039
:10070E000375280A305902E120741F552E600353D9
:10071E00DAFE752906741F552E700375290AD0F05E
:10072E00D0E0D0D0C2D3D2AF327901E14F7903E11C
:10073E004F790AE14F791EE14F7964E14F79C8E1B3
:10074E004F7817E4D5E0FDD8FAD9F6227A147B78E3
:10075E000207767A107B8C0207767A0D7BB402073D
:10076E00767A0B7BC8020776AC257525017902B225
:10077E0075E4C292D5E0FDE5256002C293D5E0FD99
:10078E00D293D5E0FDD292D5E0FDE525600A207525
:10079E0002C297307502C295E56DD5E0FD20750257
:1007AE00D297307502D2957496D5E0FDD9C1EAF88C
:1007BE00D5E0FDD8FBDBB1C2928C2522C37C007D37
:1007CE000075F00005F0EA33FAEB33FB50F6EB134D
:1007DE00FBEA13FAC3E9FFE8FEE89AF8E99BF95041
:1007EE0004EFF9EEF8B3EC33FCED33FDD5F0DFEDAD
:1007FE00F9ECF822E889F08A20D2D4F8A9F07B002F
:10080E0030F70B7BFFF42401F8E9F43400F9E885A6
:10081E0020F0A4ADF0F8E98520F0A4AFF0FEED2EA7
:10082E00F974003FFA7C04C3EA13FAE913F9E813EA
:10083E00F8DCF48BF030F70AE8F42401F8E9F4342C
:10084E0000F9E889F0C2D4F8A9F0227882B6040340
:10085E000208B6C3E5589401400302087E8522249F
:0D086E00E4F53FF540F541F542F543F5484E
:10087B000208B67882E6FC754801E522F523783844
:10088B0079C7AA3BAB3CC3EB13FBEA13FAEC14603E
:10089B0013C3EB13FBEA13FAEC14146007C3EB134B
:1008AB00FBEA13FA1207CA883F894022E5486034F5
:1008BB00C3E53F9523F8E5409400F9500CC3E89449
:1008CB0080E994FF40160208EBC3E8947FE994009B
:1008DB0050030208EB787F79000208EB788079FFF0
:1008EB008844894522E5486058E5442541F8E545AB
:1008FB003542F9854520E4300701F43543FA30E7FA
:10090B0009C3EA94F0401502092DC3EA940F500372
:10091B0002092D78FF79FF7A0F02092D78007900F3
:10092B007AF0C3E524955C5006E52460092146E581
:10093B004520E70D2146E54530E706884189428A87
:10094B004322E54870030209B0789EE6FAC3E544FA
:10095B0033F8E54533F91102E930E70BC3E894802E
:10096B00E994FF40132187C3E8947FE99400500278
:10097B002187787F79002187788079FFE820E71538
:10098B00C3E52398F84009C3E8940140030209AE7C
:10099B0078010209AEE8F424012523F8400302098B
:1009AB00AE78FF884622E5487003020A12789FE66C
:1009BB00FAA842A9431102E930E70CC3E89401E914
:1009CB0094FF40160209E9C3E894FFE99400500331
:1009DB000209E978FF79000209E9780179FFE9203A
:1009EB00E715C3E54698F84009C3E89401400302B4
:1009FB000A107800020A10E8F424012546F8400397
:100A0B00020A1078FF8824227883E6F520120F5013
:100A1B0075E890E5E820ECF0A8BDA9BE120FE875CB
:100A2B006855756900C3740013FD745513FC745538
:100A3B002CFC74003DFDECFAEDFBC3E89AE99B40FE
:100A4B0014E5682455F568E5693400F569EA2CFA74
:100A5B00EB3DFB80E5AE68AF69C3E56913F9E5686B
:100A6B0013F8C3E913F9E813F8E56828F566E569A7
:100A7B0039F5677A03C3E913F9E813F8DAF7AA2013
:100A8B001A7009756800756900020AA71AEA6008EE
:100A9B00EE28FEEF39FFDAF88E688F692275E89041
:100AAB00227883E6FFE5E820ECF7A8BDA9BE056A2E
:100ABB00C3E56A94084052756A00E97007E56B60FC
:100ACB001B020ADBC3E8956B6010E56B5006600CEC
:100ADB0014020AE70460F9020AE7E56BF56BC394AD
:100AEB006DF84021755CC0C3E89404F84017755C41
:100AFB0080C3E89404F8400D755C40C3E89404F897
:100B0B004003755C0075BB0822EFC39401601BC3E7
:100B1B00E894FFE994035012C3E89568E99569508E
:100B2B0009E55C600C155C020B3CE55CF4600205AE
:100B3B005CA85CC3E524985002A8248825C3E5254E
:100B4B00955D400B855D25E55DF46003855D5CC3BC
:100B5B00E56AB4070375BB1022306102783230624C
:100B6B00027878E52C5406601FE879A187F0A4C5BC
:100B7B00F0A2F733F8C3E8955C4002A85C882288A2
:100B8B00248825306102885E22788FE6FFC3EF94BC
:100B9B00055018C3EF94045020C3EF94035028C39F
:100BAB00EF94025030C3EF940150387533A0753475
:100BBB000F75353C75360561FC7533C07534127590
:100BCB00354075360661FC7533707534177535D045
:100BDB0075360761FC75334C75341D7535C4753628
:100BEB000961FC7533287534237535B875360B617F
:100BFB00FC85334F853450753B00753C0822A84F5C
:100C0B00A950020C14A849A94A759100C3E498F5A0
:100C1B0094E499F595759104D25875C820A8CCA980
:100C2B00CD75C824AA39AB3A8839893AC3E89AF802
:100C3B00E99BF9AA3BAB3CC3EB13FDEA13FCC3EDF9
:100C4B0013FDEC13FCC3EA9CFAEB9DFBEA28FAEBD1
:100C5B0039FB8A3B8B3C400122753BFF753CFF22E5
:0F0C6B00305802816B759100C3E4954BF594E40A
:100C7A00954CF595759104D258227892E6FF7E102C
:100C8A00305B027F053063047F037E00A93CA83BEA
:100C9A007A04C3E913F9E813F8DAF7C3E89EF8E926
:100CAA009400F94009C3E89402E9940050047802D8
:100CBA00E4F9E9FBE8FAC3E913FDE813FCC3EF948E
:100CCA0003602EEF20E00DE82CF8E93DF9ECFAED8F
:100CDA00FB020CE8E828F8E939F97A02E4FBC3EFE9
:100CEA009403400D8A4D8B4E8849894A8C4B8D4C12
:100CFA0022884D894E8A498B4A8C4B8D4C2230581A
:100D0A0002A108759100C3E4953BF594E4953CF57E
:100D1A0095759104D25822753E00752000020D3057
:100D2A00753E00752040D2AF053E20580122759DC0
:100D3A0000E53CC313C313F8086030306A06C313D6
:100D4A00C313F808C3E8940A4002780A306D08C34E
:100D5A00E8940440027804C3E53C9408400D759D6C
:100D6A0002C3E53C94104003759D03205803D2AF9B
:100D7A00227918206D027908D2AF0000C2AF205A3A
:100D8A000A7914206D027907306FE03063027978AE
:100D9A00C3E58B9940D5E59BF45440B52002A130B8
:100DAA00D8C9D2AF22C25B789CE6146007E53E142C
:100DBA007002D25B30630B05382058107538000278
:100DCA000DD6205807158115810217352275910015
:100DDA00C3E4954DF594E4954EF595759104D25872
:100DEA0022AE25305B4F78A3E6FFBF010BD25C75BC
:100DFA002500D297D295D2939170305C0375250065
:100E0A00305802C104BF020BD25C752500D297D2BA
:100E1A0095D29378A2B6010D9170305C03752500C6
:100E2A00305802C124BF030BD25C752500D297D279
:100E3A0095D293B1D7305C03752500305802C13F73
:100E4A00305B04C25C8E2522C2AFC292206A0302C2
:100E5A000E74900305206C12306E0F207502C29436
:100E6A00307502C2967419D5E0FD207502D296300B
:100E7A007502D294759F13753D02D2AF22C2AF207C
:100E8A006A03020EA99002C4306E17C2922075023C
:100E9A00C294307502C2967419D5E0FD020EAC9068
:100EAA0001C5207502D295307502D297305A06E5EF
:100EBA00256002C293207503759F10307503759FD4
:100ECA0011753D03D2AF22C2AF207502C2963075AA
:100EDA0002C294206A03020EF3900283206C0A3045
:100EEA006E07C2927419D5E0FD207502D29430754E
:100EFA0002D296207503759F11307503759F107580
:100F0A003D04D2AF22C2AF206A03020F31900242DF
:100F1A00306E17207502C296307502C294C292745E
:100F2A0019D5E0FD020F349001B3D293305A0EE581
:100F3A0025600A207502C297307502C295759F1303
:100F4A00753D05D2AF22C2AF207502C29430750238
:100F5A00C296206A03020F7A9001F1206C12306E59
:100F6A000F207502C296307502C2947419D5E0FD3D
:100F7A00D292207503759F10307503759F11753DC8
:100F8A0006D2AF22C2AF206A03020FB890035630CE
:100F9A006E1F207502C296307502C294207502C275
:100FAA0094307502C2967419D5E0FD020FBB900108
:100FBA00D7207502D297307502D295305A0EE525A0
:100FCA00600A207502C295307502C29720750375B2
:100FDA009F11307503759F10753D01D2AF229001A4
:100FEA00B1D297D295D293C296C294C29222C3E545
:100FFA004F9535E55095365001227890E6FFC3EFBC
:10100A0094055018C3EF9404501BC3EF9403501E69
:10101A00C3EF94025021C3EF94015024C3E54F94C7
:10102A003CF8021053C3E54F9428F8021053C3E565
:10103A004F941AF8021053C3E54F9412F802105352
:10104A00C3E54F940AF8021053E5509400F9884F0B
:10105A0089502230580302105D2278807607788101
:0E106A007607788276017884760378837601A3
:1010780078867609788F7601789076057895760265
:1010880078927603789B760D789376067887760142
:10109800789C76027888760178897601788576005A
:1010A800788C7601788D7600788E76B47896762569
:1010B800789776D078987678789976C8789A7604FA
:1010C800789D7600227893E6FF756409756501C3FB
:1010D800BF0209756405756501021112C3BF0309D2
:1010E800756405756502021112C3BF0409756405AC
:1010F800756503021112C3BF050675640975650796
:10110800C3BF06067564007565007887E6FFC26C84
:10111800C3BF0302D26CC26BC3BF0402D26BC26AE4
:101128007418552D6002D26AC26E6002D26ED26FF8
:101138006002C26FC2757888E630E102D275C27665
:101148007889E630E102D276C3EF94026008758EA2
:1011580001D26D021163758E00C26D227880E6148B
:1011680090008093789EF67881E6149000809378BA
:101178009FF6120FE822789BE61490008D9378A0D2
:10118800F6120FE8227886E61490009A9378A1F672
:10119800120FE822789CE6149000A79378A2F678BC
:1011A8009CE6149000AC9378A3F6120FE8222278FC
:1011B80096E6FA7897E6FB3077047A007BFFC3EB74
:1011C8009AFCC3948250027C82756C00056CEC8595
:1011D8006CF0A4C3E5F0948040F222C2D353D9BF87
:1011E8007581C043FF8012073775EF0243B203E5EC
:1011F800B324044002F5B37580FF75A40075F1B2FD
:1012080075D4DF7590A975A5FC75F2FE75D50175C5
:10121800A60175E241120FE8E4F8F6D8FD11641250
:10122800176511CD3164317E318D319C31B631B7BE
:101238007898866D120FE875885075890275C824EC
:1012480075910475D84012074B12075A12074312BA
:101258000761120743120768120743121CE51207B9
:101268004B12074B12074775A82275B80275E6900E
:1012780075F610759B80759D0375D10E75BC5875F4
:10128800BB0875BA1175E880120737D2AF120A1376
:1012980043DA01C2D8C26912074B753001D2597AB4
:1012A80005E55770027A0512073BE558C3940240DA
:1012B800EEE52E541F855A59F55AB559E2DAE2C2BD
:1012C8005953DACF20760343DA2030760343DA1015
:1012D800C2D8C26912074712073B7802741F552EFD
:1012E80070027800C3E5589840EDC2AF12075A1251
:1012F800075A12075AD2AF12074B75470012073B1D
:10130800788CE6C3940150030213CEE530C39401F0
:1013180050030213CE741F552E6035C3E55894FF51
:1013280050030213CEC2AF12076FD2AF120747C3E2
:10133800E558940150EFC2AF12075A12073F12073F
:101348005AD2AF120747C3E55894FF40E9021D6A15
:101358007F05D27731B7120747C2AFC27731B7C31B
:10136800E558947FD2AF4068C2AF12076FD2AFDFA3
:10137800E1C3E55894057897F612074B1218141232
:101388001CED7F0AD27731B7120747C2AFC2773157
:10139800B7C3E558947FD2AF50E8C2AF12075A12CC
:1013A800073F12075AD2AFDFDBE55824057896F6D7
:1013B80012074B121814121D1C120747C3E5589444
:1013C800FF40F6021D6AC3E5589547400385584714
:1013D800120747C3E558940140026105C2AF1207DE
:1013E8006F12076F12076FD2AF12074B753000E408
:1013F800F531F5320531E531F470360532789AE683
:101408007828146012785014600D78A01460087859
:10141800F0146003753200C3E53298401415327831
:1014280099866DC2AF12076FD2AF7898866D120792
:101438004712073BE5287008741F552E700241A516
:10144800C3E558940640AD120747E5287003021219
:10145800A5120FE8E4F522F523F524F525755CFFC0
:0E1468007885865FF53FF540F541F542F54386
:10147600F56AF548F52BF52CF55B120B94756A08A1
:1014860075BB10120737120AA8E5E820ECFBA8BDC9
:10149600A9BEE97001F8886B120AAC756A0875BBBB
:1014A600107895E630E0030214EC7887E6FE7602C3
:1014B60011CD7887EEF6D261C2AF120B6485225C3D
:1014C60085225DD2AFC26175250075620075630124
:1014D600D260D263753800120F50120F8E120C10A4
:1014E600120B9402161B7887E6FE76037893E6FDC8
:1014F600760511CD7887EEF67893EDF6D260D26157
:10150600D26E120F50120F8E120B64120737120E84
:1015160052120737120737120E8712073B120ED1E7
:1015260012073B12073B120F0F12073F120F501202
:10153600073B120737C261D262120AA8120AAC121E
:101546000B64756A0875BB10120F8E120C09120C0B
:1015560084120FF8115D120E52120C09120C84122D
:101566000FF8115D120E87120C09120C84120FF877
:10157600115D120ED1120C09120C84120FF8115DB6
:10158600120F0F120C09120C84120FF8115D120FB4
:1015960050120C09120C84120FF8C3E54F9535E56D
:1015A600509536400C115DC3E5589401508B0217D7
:1015B60035115DC2627887E6FE760211CD7887EE38
:1015C600F685225C855E5D855E2575620075630124
:1015D600D263753800C2AF207502C296307502C25A
:1015E60094207502C294307502C296742DD5E0FD22
:1015F600D2AF120F8E120C10120C6B120C84120D3D
:1016060008756A0075BB0802161B11CD120F8E7580
:101616006A0075BB08120D2A120DAF120DD71208FB
:1016260059120DEB120E52120C10120C6B120C8486
:10163600120D08120D21120DAF120DD71208B71296
:101646000DEB120E87120C10120C6B120C84120D7D
:1016560008120D2A120DAF120DD71208F0120DEB5B
:10166600120ED1120C10120C6B120C84120D0812F1
:101676000D21120DAF120DD712094D120DEB120FDF
:101686000F120C10120C6B120C84120D08120D2A7C
:10169600120DAF120DD71209B1120DEB120F501227
:1016A6000C10120C6B120C84120D08120D21120A6A
:1016B600A8120DAF120DD7120AAC120DEB120F8E37
:1016C600120C10120C6B120C84120D0830632A8552
:1016D6005E5C855E5D756200756301C3E538946482
:1016E600400AC263D2647537140216FFC3E55894E4
:1016F60001400302161B021735306419E5371470D2
:1017060005C264021610F537C3E55894014003027A
:10171600161B021735C3E55B94FA5013741F552E3A
:101726007004E5286009C3E53C94F05002C11B1221
:101736000FE87887E6FE760211CD7887EEF6E4F5B7
:1017460022F523F524F525F55FC260120737120F3F
:10175600E8741F552E7006E528700241A561F790C2
:101766001A0D7820121C00E520B4550CA3121C009B
:10177600E520B4AA0302178611641218140218137E
:10178600901A037880121C00A308121C00A30812EA
:101796001C00901A067883121C00A308121C00A3D2
:1017A60008A308121C00A308121C00A308121C00A0
:1017B600A308121C00A308A308A308121C00A30870
:1017C600A308121C00A308121C00A308121C00A3E5
:1017D60008A308121C00A308121C00A308A30812E1
:1017E6001C00A308121C00A308121C00A308121C4C
:1017F60000A308121C00A308121C00A308121C0058
:10180600A308121C00A308121C00901A2122C2AFC2
:10181600121C3F121C19901A00740A121C05A3749C
:1018260004121C05A37410121C05901A037880126A
:101836001C04A308121C04A308121C04901A0678A0
:1018460083121C04A308121C04A308A308121C0478
:10185600A308121C04A308121C04A308121C04A348
:0F18660008A308A308121C04A308A308121C045B
:10187500A308121C04A308121C04A308A308121C25
:1018850004A308121C04A308A308121C04A308122D
:101895001C04A308121C04A308121C04A308121C90
:1018A50004A308121C04A308121C04A308121C0498
:0F18B500A308121C04121C52121C30901A21227C
:101A00000A04100909040103FF0901010155AA0193
:101A1000FFFF0105FF0306FF0225D02850040D0239
:021A200000FFC5
:101A4000235475726E69677933304123202020203A
:101A500023424C48454C4923463333302320202031
:101A60002020202020202020202020202020202076
:101C0000E493F622E6438F01538FFD75EF0275B71B
:101C1000A575B7F1F0538FFE22438F02438F0175F4
:101C2000EF0275B7A575B7F1901A0DF0538FFC222E
:101C3000901A0D74559105901A0E74AA9105227A86
:101C40003079D07820901A409100E520F709A3DA86
:101C5000F7227A3079D0901A40E7910509A3DAF992
:101C600022AB6EA86FBB01057980021CE2BB0205A6
:101C70007981021CE2BB03057982021CE2BB0405E8
:101C80007984021CE2BB05057983021CE2BB0605D0
:101C90007995021CE2BB07057986021CE2BB0805A8
:101CA000798F021CE2BB09057990021CE2BB0A0590
:101CB0007992021CE2BB0B05799B021CE2BB0C056E
:101CC0007993021CE2BB0D057987021CE2BB0E056D
:101CD000799C021CE2BB0F057988021CE27989021B
:101CE0001CE2E8F7227C0512074BDCFB22C2AF1294
:101CF000075A12076112076812076F12073F12078F
:101D00005A12076112076812076F12073F12075A2B
:101D100012076112076812076FD2AF22C2AF120713
:101D20006F12076812076112075A12073F12076FF6
:101D300012076812076112075A12073F12076F1243
:101D4000076812076112075AD2AF22AE6EAF6FC298
:101D5000AF12075A12075A12075A12073FDEF21241
:101D6000076F12073FDFF8D2AF2291ED91E591E5C1
:101D7000756E01756F01757000B14B7C05AD581221
:101D8000074BC3ED955870F5C3E55894014009C35E
:101D9000E55894FF4032A1A6916112181491EDC24A
:101DA000AF75EF1291E5DCD50570C3E57094035073
:101DB0000280C691E5056FE56E149000B193F808B6
:101DC000C3E56F98500280AE91E591E5056EC3E5DD
:101DD0006E94115002809C121064121814C2AF75D8
:041DE000EF1291E588
:00000001FF
